:020000040000FA
:06000000ADEF04F0120058
:0600080036EF02F01200C9
:06001800C2EF00F012002F
:06002A000100780900004E
:080030000A0F000002000000AD
:08003800D9CFE6FFE1CFD9FFAB
:100040008C808C828C848C868C888C8A8C8C8C8E18
:100050008A868D808D828D848D868D888D8A8D8C0B
:100060008D8E8A8A8E808E828E848E868E888E8AEF
:100070008E8C8E9E8A9889808982898489868F80D9
:100080008F828F848F868A808A828A8495909592C7
:10009000959495969598959A959C959E93969690FD
:1000A0009692969496969698969A969C969E939AE1
:1000B00097909792979497969798979A979C979ED0
:1000C00093989290929292949296989098929894F3
:1000D000989693909392939482888286949082804B
:1000E0000201006B0051006E016AD890015004E6D5
:1000F000B40E005C000E015810E20051EA6A000FD5
:10010000E96E080EEA22EF6A0051EA6A000FE96E12
:100110000A0EEA22EF6A002BE5D7006B230E005D82
:1001200017E20051EA6A000FE96E040EEA22EF6A54
:100130000051EA6A000FE96E010EEA22EF6A0051EF
:10014000EA6A230FE96E010EEA22EF6A002BE6D776
:10015000FE0EDBCFE6FF0DDAE552850EE66E71ECA2
:1001600004F0E552200EBE6E030EBF6EB196B19C38
:100170009E949D849F9494940B0EBD6EE552E7CFA0
:10018000D9FF1200DACFE4FFE2CFDAFFE9CFE4FFD4
:10019000EACFE4FFE65202010151066E076A800EC3
:1001A000061801E1075001E084D0006B230E005DCA
:1001B00013E20051EA6A230FE96E010EEA22EF50C2
:1001C000E66E0051EA6A000FE96E010EEA22E5527E
:1001D000E750EF6E002BEAD7016B0101005101E0FF
:1001E0008C90015101E08C92025101E08C940351FA
:1001F00001E08C96045101E08C98055101E08C9A45
:10020000065101E08C9C075101E08C9E085101E0F1
:100210008D90095101E08D920A5101E08D940B51AE
:1002200001E08D960C5101E08D980D5101E08D9A01
:100230000E5101E08D9C0F5101E08D9E105101E0A7
:100240008E90115101E08E92125101E08E94135163
:1002500001E08E96145101E08E98155101E08E9ABE
:10026000165101E08E9C175101E08E9E185101E05D
:100270008A96195101E08A9A1A5101E08A981B5115
:1002800001E089901C5101E089921D5101E089949F
:100290001E5101E089961F5101E08F90205101E02D
:1002A0008F92215101E08F94225101E08F96010E2F
:1002B000466F020101510101005D01E18C800201E4
:1002C00001510101015D01E18C8202010151010135
:1002D000025D01E18C84020101510101035D01E134
:1002E0008C86020101510101045D01E18C8802014B
:1002F00001510101055D01E18C8A020101510101F9
:10030000065D01E18C8C020101510101075D01E1F3
:100310008C8E020101510101085D01E18D80020115
:1003200001510101095D01E18D82020101510101CB
:100330000A5D01E18D840201015101010B5D01E1C2
:100340008D860201015101010C5D01E18D880201E0
:10035000015101010D5D01E18D8A0201015101018F
:100360000E5D01E18D8C0201015101010F5D01E182
:100370008D8E020101510101105D01E18E800201AB
:1003800001510101115D01E18E8202010151010162
:10039000125D01E18E84020101510101135D01E151
:1003A0008E86020101510101145D01E18E88020176
:1003B00001510101155D01E18E8A02010151010126
:1003C000165D01E18E8C020101510101175D01E111
:1003D0008E8E020101510101185D01E18A86020140
:1003E00001510101195D01E18A8A020101510101F6
:1003F0001A5D01E18A880201015101011B5D01E1E1
:1004000089800201015101011C5D01E18982020123
:10041000015101011D5D01E18984020101510101C8
:100420001E5D01E189860201015101011F5D01E1AB
:100430008F80020101510101205D01E18F820201E3
:1004400001510101215D01E18F840201015101018E
:10045000225D01E18F860201012B9E94E552E5CFDA
:10046000EAFFE5CFE9FFE5CFDAFF1100DACFE4FFDD
:10047000E2CFDAFFE9CFE4FFEACFE4FFF6CFE4FF13
:10048000F7CFE4FFF5CFE4FFF3CFE4FFF4CFE4FFD1
:10049000FACFE4FF00EE04F0020EE80403E3EECF2F
:1004A000E4FFFBD700EE00F0040EE80403E3EECF18
:1004B000E4FFFBD7E652C7BA13D0C9CFB4FAC7A43A
:1004C0000BD0B6CAE6FF70D8E552C96E0A01010E1C
:1004D000B76F030EB56F03D00A01010EB56F23D0BD
:1004E0000A01B50506E1C9CFB6FA020EB56FB76BC2
:1004F0001AD0020EB55D0BE1C950E66EB651B725B4
:10050000E66E72D8E552E5520A01B72B0CD0030E05
:10051000B55D09E1B651B725E66E46D8E552C96E1C
:10052000C6880A01B72BC6889E96E55200EE03F0F6
:10053000040EE80403E3E5CFEDFFFBD700EE05F082
:10054000020EE80403E3E5CFEDFFFBD7E5CFFAFFAA
:10055000E5CFF4FFE5CFF3FFE5CFF5FFE5CFF7FFFC
:10056000E5CFF6FFE5CFEAFFE5CFE9FFE5CFDAFF1C
:100570001100D9CFE6FFE1CFD9FFFE0EDB50C86EE8
:10058000C00EE66E060EE66E92EC04F0E552E55201
:10059000D08EF28EF28C9E969D869F86C580C688F0
:1005A000E552E7CFD9FF1200D9CFE6FFE1CFD9FF5F
:1005B000FE0EDB50006E016AD890015004E6B40EC6
:1005C000005C000E01580AE2FE0EDB50EA6A000FE2
:1005D000E96E080EEA22EF5003D002D0000E00D0E0
:1005E000E552E7CFD9FF1200D9CFE6FFE1CFD9FF1F
:1005F000FE0EDB50EA6A000FE96E080EEA22FD0EDD
:10060000DBCFEFFFFE0EDB50EA6A000FE96E0A0E49
:10061000EA22010EEF6EE552E7CFD9FF1200D38830
:10062000D38AD38C9B8CB00EE66E06DDE5520A01B0
:10063000915101E1E0D00601016B026B036B046B89
:10064000180E0601015D000E0259000E0359000E3E
:10065000045931E2000E06010125E96E0A0E060179
:100660000221EA6EEF5020E09D96000E0601012562
:10067000E96E080E06010221EA6EEF50E66E000EEA
:1006800006010125E96E040E06010221EA6EE5521B
:10069000E750EF6E9D86000E06010125E96E0A0EF9
:1006A00006010221EA6EEF6A0601012B000E022309
:1006B00003230423C5D70601920E016F026B036B5F
:1006C000046B950E0601015D000E0259000E0359E0
:1006D000000E04593FE2000E06010125E96E0A0EE4
:1006E00006010221EA6EEF502EE09D96000E0601F3
:1006F0000125E96E080E06010221EA6EEF50E66E52
:1007000001C600F002C601F003C602F004C603F001
:100710007A0E005E000E015A000E025A000E035AB5
:10072000000E0024E96E040E0120EA6EE552E75047
:10073000EF6E9D86000E06010125E96E0A0E060188
:100740000221EA6EEF6A0601012B000E0223032349
:100750000423B7D70601A40E016F026B036B046B71
:10076000AC0E0601015D000E0259000E0359000E89
:1007700004593FE2000E06010125E96E0A0E06014A
:100780000221EA6EEF502EE09D96000E0601012533
:10079000E96E080E06010221EA6EEF50E66E01C610
:1007A00000F002C601F003C602F004C603F0890E91
:1007B000005E000E015A000E025A000E035A000E8F
:1007C0000024E96E040E0120EA6EE552E750EF6E58
:1007D0009D86000E06010125E96E0A0E0601022122
:1007E000EA6EEF6A0601012B000E022303230423A5
:1007F000B7D70A01916B0201006B230E0201005D65
:1008000018E29D9602010051EA6A000FE96E040E9B
:10081000EA22EF50E66E02010051EA6A230FE96E08
:10082000010EEA22E552E750EF6E9D860201002B91
:10083000E4D70101466B00000101460501E0FCD749
:04084000F6D61200D6
:0C0844002A0EF66E000EF76E000EF86E25
:100850000F010900F550056F0900F550066F03E11F
:10086000056701D03DD00900F550006F0900F55033
:10087000016F0900F550026F09000900F550E96E9B
:100880000900F550EA6E090009000900F550036FF0
:100890000900F550046F09000900F6CF07FFF7CFF4
:1008A00008FFF8CF09FF00CFF6FF01CFF7FF02CF17
:1008B000F8FF0F01035302E1045307E00900F5506C
:1008C000EE6E0307F8E20407F9D707CFF6FF08CF6B
:1008D000F7FF09CFF8FF0F010507000E065BBFD732
:0208E000120004
:0E08E200D9CFE6FFDACFE6FFE1CFD9FFE2CFB4
:1008F000DAFFFD0EDB507E0BCD6EFD0EDBAC02D0C1
:10090000CD8E01D0CD9ECF6ACE6A9E90DBAE02D056
:100910009D8001D09D90CD80E552E5CFDAFFE7CFF5
:04092000D9FF1200E9
:0C092400D9CFE6FFDACFE6FFE1CFD9FF24
:10093000E2CFDAFF3F0EC716C66AC56AFD0EDB506E
:10094000C612FC0EDB50C71294869488C68AE55204
:0A095000E5CFDAFFE7CFD9FF120070
:06095A001EEE00F02EEE7F
:1009600000F0F86A059C22EC04F0BBEC04F00FECFC
:0609700003F0FBD71200AA
:0209760012006D
:0209780000007D
:020000040030CA
:0100010008F6
:0100020018E5
:010003001EDE
:010006008178
:00000001FF
